:100000000C9438000C9453000C9453000C9453003F
:100010000C9453000C9453000C9453000C94530014
:100020000C9453000C9453000C9453000C94530004
:100030000C9453000C9453000C9453000C945300F4
:100040000C9453000C94BB020C9453000C9453007A
:100050000C94B40E0C9453000C9453000C94530065
:100060000C9453000C9453000C9453000C945300C4
:1000700011241FBECFEFD4E0DEBFCDBF12E0A0E061
:10008000B1E0ECE5F2E202C005900D92AC3FB107A1
:10009000D9F713E0ACEFB2E001C01D92A93EB10761
:1000A000E1F70C9472000C940000CF93DF93CDB76E
:1000B000DEB7E4E3F0E08FEF8083EAE3F0E08EE286
:1000C0008083ABE3B0E0EBE3F0E0808182608C936F
:1000D000ABE3B0E0EBE3F0E0808180628C93DF91F2
:1000E000CF910895CF93DF93CDB7DEB70E9455002F
:1000F0000E94AC020E94B20D7894A5E3B0E0E5E363
:10010000F0E0808181608C930E947F020E9428062B
:100110000E94F7020E9441030E948B030E94D503B4
:100120000E941F040E9469040E94B30400C08091D1
:10013000FE02813031F41092FE020E9494100E945F
:10014000A31080910B038130E1F4A5E3B0E0E5E377
:10015000F0E0808184608C930E94BE0C0E94460F68
:100160000E94C8060E94DD070E9411090E947405C2
:100170000E945906A5E3B0E0E5E3F0E080818B7FC3
:100180008C938091FC02813091F61092FC020E94C7
:10019000FD04CDCFCF93DF93CDB7DEB764E084E02D
:1001A0000E94E7006CE480E00E94E7001092FE02EB
:1001B0008091FE028823E1F36AE08CE60E94E7006A
:1001C00060E085E00E94E700DF91CF910895CF9332
:1001D000DF93CDB7DEB724970FB6F894DEBF0FBE1E
:1001E000CDBF8B836C83ABE3B0E0EBE3F0E08081C9
:1001F0008D7F8C9387E08A8340C0ABE3B0E0EBE374
:10020000F0E08081877F8C930000000000000000F8
:100210008A81282F332727FD309581E090E0022E38
:1002200002C0880F991F0A94E2F7982F8B818923C7
:1002300089838981882341F0ABE3B0E0EBE3F0E010
:10024000808184608C9307C0ABE3B0E0EBE3F0E027
:1002500080818B7F8C930000000000000000ABE3E6
:10026000B0E0EBE3F0E0808188608C930000000058
:10027000000000008A8181508A838A8188230CF0E3
:10028000BCCF87E08A8340C0ABE3B0E0EBE3F0E0B3
:100290008081877F8C9300000000000000008A812D
:1002A000282F332727FD309581E090E0022E02C0F1
:1002B000880F991F0A94E2F7982F8C8189238983EC
:1002C0008981882341F0ABE3B0E0EBE3F0E080818B
:1002D00084608C9307C0ABE3B0E0EBE3F0E0808197
:1002E0008B7F8C930000000000000000ABE3B0E0C7
:1002F000EBE3F0E0808188608C9300000000000058
:1003000000008A8181508A838A8188230CF0BCCFC7
:10031000ABE3B0E0EBE3F0E08081877F8C93ABE36D
:10032000B0E0EBE3F0E080818B7F8C93ABE3B0E057
:10033000EBE3F0E0808182608C9324960FB6F89412
:10034000DEBF0FBECDBFDF91CF910895CF93DF9376
:10035000CDB7DEB724970FB6F894DEBF0FBECDBF82
:100360008C83ABE3B0E0EBE3F0E080818D7F8C9396
:1003700087E08A834CC0ABE3B0E0EBE3F0E0808140
:10038000877F8C9300000000000000000000000048
:10039000000000008A81282F332727FD309581E057
:1003A00090E0022E02C0880F991F0A94E2F7982F5E
:1003B0008C8189238B838B81181644F4ABE3B0E0E6
:1003C000EBE3F0E0808184608C9307C0ABE3B0E0A6
:1003D000EBE3F0E080818B7F8C9300000000000055
:1003E00000000000000000000000ABE3B0E0EBE321
:1003F000F0E0808188608C93000000000000000025
:1004000000000000000000008A8181508A838A81F8
:1004100088230CF0B0CF1B82ABE3B0E0EBE3F0E05D
:100420008081877F8C9300000000000000000000A6
:1004300000000000000087E08A833DC0ABE3B0E02D
:10044000EBE3F0E0808188608C93E9E3F0E0808169
:1004500089838981992780719070181619068CF408
:100460008A81282F332727FD309581E090E0022EE6
:1004700002C0880F991F0A94E2F7982F8B81892B6D
:100480008B8300000000000000000000000000005E
:100490000000ABE3B0E0EBE3F0E08081877F8C937A
:1004A000000000000000000000000000000000004C
:1004B0008A8181508A838A8188230CF0BFCFABE385
:1004C000B0E0EBE3F0E08081877F8C93ABE3B0E0BA
:1004D000EBE3F0E080818B7F8C93ABE3B0E0EBE368
:1004E000F0E0808182608C938B81992724960FB6EF
:1004F000F894DEBF0FBECDBFDF91CF910895CF93AB
:10050000DF93CDB7DEB70E94CA001092FC02809143
:10051000FC028823E1F30E943A050E94E30A10924C
:10052000FC028091FC028823E1F31092FC0280918E
:10053000FC028823E1F31092FC0264E084E00E9454
:10054000E7006CE480E00E94E7000E94FD040E9446
:100550009305DF91CF910895CF93DF93CDB7DEB7A9
:10056000E3E5F0E082E08083E9E5F0E082E080838B
:10057000DF91CF9108951F920F920FB60F92112421
:100580008F93CF93DF93CDB7DEB7809100038F5F5A
:100590008093000380910003883409F581E0809303
:1005A000FF02109200038091A4038F5F8093A40345
:1005B0008091A403843629F41092A40381E08093EF
:1005C000FC028091A3038F5F8093A3038091A30318
:1005D0008A3029F41092A30381E08093FE02DF9118
:1005E000CF918F910F900FBE0F901F901895CF93C2
:1005F000DF93CDB7DEB762E480E00E94E70010929F
:10060000FC028091FC028823E1F31092FC026CE56D
:1006100089E00E94E7001092FE028091FE0288238A
:10062000E1F31092FE021092A50316C08091A5037B
:10063000682F8AE00E94E7008091A5039927FC01BA
:10064000E95CFE4F8081682F8BE00E94E70080917B
:10065000A5038F5F8093A5038091A503863330F3B4
:1006600060EA88E00E94E7001092FE028091FE029C
:100670008823E1F36CE480E00E94E700DF91CF91F2
:100680000895CF93DF93CDB7DEB762E480E00E9498
:10069000E7001092FC028091FC028823E1F31092A3
:1006A000FC026DE589E00E94E7001092FE02809155
:1006B000FE028823E1F31092FE021092A50316C0F9
:1006C0008091A503682F8AE00E94E7008091A5032E
:1006D0009927FC01E958FE4F8081682F8BE00E942A
:1006E000E7008091A5038F5F8093A5038091A50308
:1006F000863330F360EA88E00E94E7001092FE0241
:100700008091FE028823E1F36CE480E00E94E70020
:10071000DF91CF910895CF93DF93CDB7DEB762E439
:1007200080E00E94E7001092FC028091FC02882386
:10073000E1F31092FC026EE589E00E94E70010925E
:10074000FE028091FE028823E1F31092FE021092D5
:10075000A50316C08091A503682F8AE00E94E700D8
:100760008091A5039927FC01E954FE4F8081682FF1
:100770008BE00E94E7008091A5038F5F8093A50323
:100780008091A503863330F360EA88E00E94E70099
:100790001092FE028091FE028823E1F36CE480E077
:1007A0000E94E700DF91CF910895CF93DF93CDB7FB
:1007B000DEB762E480E00E94E7001092FC028091C4
:1007C000FC028823E1F31092FC026FE589E00E94AD
:1007D000E7001092FE028091FE028823E1F310925E
:1007E000FE021092A50316C08091A503682F8AE02F
:1007F0000E94E7008091A5039927FC01E950FE4F74
:100800008081682F8BE00E94E7008091A5038F5FB5
:100810008093A5038091A503863330F360EA88E0D6
:100820000E94E7001092FE028091FE028823E1F30D
:100830006CE480E00E94E700DF91CF910895CF93B0
:10084000DF93CDB7DEB762E480E00E94E70010924C
:10085000FC028091FC028823E1F31092FC0260E626
:1008600089E00E94E7001092FE028091FE02882338
:10087000E1F31092FE021092A50316C08091A50329
:10088000682F8AE00E94E7008091A5039927FC0168
:10089000E95CFD4F8081682F8BE00E94E70080912A
:1008A000A5038F5F8093A5038091A503863330F362
:1008B00060EA88E00E94E7001092FE028091FE024A
:1008C0008823E1F36CE480E00E94E700DF91CF91A0
:1008D0000895CF93DF93CDB7DEB762E480E00E9446
:1008E000E7001092FC028091FC028823E1F3109251
:1008F000FC0261E689E00E94E7001092FE0280910E
:10090000FE028823E1F31092FE021092A50316C0A6
:100910008091A503682F8AE00E94E7008091A503DB
:100920009927FC01E958FD4F8081682F8BE00E94D8
:10093000E7008091A5038F5F8093A5038091A503B5
:10094000863330F360EA88E00E94E7001092FE02EE
:100950008091FE028823E1F36CE480E00E94E700CE
:10096000DF91CF910895CF93DF93CDB7DEB762E4E7
:1009700080E00E94E7001092FC028091FC02882334
:10098000E1F31092FC0262E689E00E94E700109217
:10099000FE028091FE028823E1F31092FE02109283
:1009A000A50316C08091A503682F8AE00E94E70086
:1009B0008091A5039927FC01E954FD4F8081682FA0
:1009C0008BE00E94E7008091A5038F5F8093A503D1
:1009D0008091A503863330F360EA88E00E94E70047
:1009E0001092FE028091FE028823E1F36CE480E025
:1009F0000E94E700DF91CF910895CF93DF93CDB7A9
:100A0000DEB789ED8093A50313C060E085E00E9406
:100A1000E7008091A503682F86E00E94E70064E567
:100A200087E00E94E7008091A5038F5F8093A50374
:100A30008091A5038C3D48F385EE8093A50313C0F8
:100A400060E085E00E94E7008091A503682F86E0C2
:100A50000E94E70064E587E00E94E7008091A5031B
:100A60008F5F8093A5038091A503883E48F3DF91B3
:100A7000CF910895CF93DF93CDB7DEB764970FB6CC
:100A8000F894DEBF0FBECDBF8DE589838EE58A83E6
:100A90008FE58B8389E48C838BE58D838DE18E8359
:100AA0008CE58F83188680E2898789E28A8786E3CE
:100AB0008B8781E48C878AE08D8781E48E8781E053
:100AC0008F8786E2888B20E1CE010196AC0162E03F
:100AD00087E00E94BE0564960FB6F894DEBF0FBE95
:100AE000CDBFDF91CF910895CF93DF93CDB7DEB720
:100AF00060E085E00E94E7006FEC86E00E94E7007E
:100B00006CE887E00E94E70061E085E00E94E70072
:100B10006BE086E00E94E7006DE887E00E94E70056
:100B2000DF91CF910895CF93DF93CDB7DEB760E02B
:100B300085E00E94E70060E286E00E94E70060E84E
:100B400087E00E94E70060E085E00E94E7006EE336
:100B500086E00E94E70064E887E00E94E70060E02A
:100B600085E00E94E7006CE586E00E94E70068E807
:100B700087E00E94E700DF91CF910895CF93DF9344
:100B8000CDB7DEB72D970FB6F894DEBF0FBECDBF41
:100B900089876A875C874B872D878A85282F33272B
:100BA0008EE190E0A901489F9001499F300D589F28
:100BB000300D112489859927820F931F98878F8381
:100BC0008D85282F33278F819885820F931F9E83D1
:100BD0008D831092A5038F8198859C838B8328C079
:100BE0008B818A838B819C81892F99278983698155
:100BF00085E00E94E7006A8186E00E94E70040915C
:100C0000A503842F99279C018B859C85F901E80F0A
:100C1000F91F8081982F842F8F5F8093A503692F00
:100C200087E00E94E7008B819C8101969C838B83E7
:100C30002B813C818D819E812817390788F22D9662
:100C40000FB6F894DEBF0FBECDBFDF91CF910895F0
:100C5000CF93DF93CDB7DEB781E091E029E0AC011F
:100C60006EE083E00E94BE05DF91CF910895CF939F
:100C7000DF93CDB7DEB722970FB6F894DEBF0FBE75
:100C8000CDBF8A838A81882321F48A818652898311
:100C900003C08A81805389838981992787FD909534
:100CA00022960FB6F894DEBF0FBECDBFDF91CF9175
:100CB00008950F931F93CF93DF93CDB7DEB72D9792
:100CC0000FB6F894DEBF0FBECDBF8091B2039091F6
:100CD000B3032EE130E0B9010E940711CB019B83E1
:100CE0008A83CE0104962A813B814AE050E0BC0110
:100CF000C9010E94D610CE010496DC01FD010190CD
:100D00000020E9F73197CF018A1B9B0B8983109252
:100D1000A5031CC08091A503082F11278091A5036E
:100D2000282F3327CE010496FC01E20FF31F8081A8
:100D30000E943706282FCE010996FC01E00FF11F13
:100D400020838091A5038F5F8093A5038091A503E5
:100D5000282F33278981992787FD909528173907F0
:100D6000CCF2298199818BE0382F391BCE0109966D
:100D7000AC016EE0832F0E94BE052D960FB6F8944D
:100D8000DEBF0FBECDBFDF91CF911F910F910895B0
:100D9000CF93DF93CDB7DEB729970FB6F894DEBFB8
:100DA0000FBECDBF8091BA039091BB038E5590408A
:100DB0009C838B838B819C8123E030E0B9010E946E
:100DC0000711CB019A83898389819A818A309105A1
:100DD00024F089E090E09A83898389819A8199231C
:100DE00014F41A8219822091040330910503898139
:100DF0009A818217930709F4D7C089819A8182303A
:100E000091052CF460E184E00E94E70004C060E0FA
:100E100084E00E94E70089819A8190930503809382
:100E2000040380E88D8384E88E8388E88F8389813A
:100E30009A8199878887888599858430910509F4F6
:100E40005FC08885998585309105DCF48885998512
:100E50008130910509F43FC08885998582309105DC
:100E60002CF488859985009779F173C088859985D8
:100E700082309105B9F18885998583309105C9F152
:100E800068C0888599858730910509F44EC08885AA
:100E90009985883091055CF4888599858530910520
:100EA000B1F18885998586309105C1F152C0888558
:100EB00099858830910509F43FC0888599858930E6
:100EC000910509F440C045C080E88D8384E88E8395
:100ED00088E88F833EC081E88D8384E88E8388E82C
:100EE0008F8337C082E88D8384E88E8388E88F8380
:100EF00030C083E88D8384E88E8388E88F8329C09F
:100F000083E88D8385E88E8388E88F8322C083E819
:100F10008D8386E88E8388E88F831BC083E88D836A
:100F200087E88E8388E88F8314C083E88D8387E801
:100F30008E8389E88F830DC083E88D8387E88E8355
:100F40008AE88F8306C083E88D8387E88E838BE8E9
:100F50008F8360E085E00E94E70060E286E00E9407
:100F6000E7008D81682F87E00E94E70060E085E060
:100F70000E94E7006EE386E00E94E7008E81682F02
:100F800087E00E94E70060E085E00E94E7006CE5F2
:100F900086E00E94E7008F81682F87E00E94E700CB
:100FA00060E084E00E94E70029960FB6F894DEBF67
:100FB0000FBECDBFDF91CF910895CF93DF93CDB713
:100FC000DEB726970FB6F894DEBF0FBECDBF809177
:100FD000AA039091AB0326E130E0B9010E9407110A
:100FE000CB0106969E838D838D819E8199230CF47F
:100FF00046C08D819E812AE030E0B9010E94071130
:10100000CB018A838D819E812AE030E0B9010E9464
:1010100007118983898186958C5F89838A81282F2E
:10102000332786E890E0821B930B9C838B8320916F
:101030000D0130910E018B819C818217930761F025
:1010400080910D0190910E010E9496088B819C81E8
:1010500069810E94D0080AC090910903898198177C
:1010600029F08B819C8169810E94D00889818093BD
:1010700009038B819C8190930E0180930D018D81DA
:101080009E8199230CF049C08D819E819095819518
:101090009F4F9E838D838D819E812AE030E0B90130
:1010A0000E940711CB018A838D819E812AE030E066
:1010B000B9010E94071189838981869589838A8174
:1010C00099278A579F4F9C838B8320910D013091E4
:1010D0000E018B819C818217930761F080910D0135
:1010E00090910E010E9496088B819C8169810E94DB
:1010F000D0080AC0909109038981981729F08B8143
:101100009C8169810E94D0088981809309038B8129
:101110009C8190930E0180930D0126960FB6F89452
:10112000DEBF0FBECDBFDF91CF910895CF93DF9388
:10113000CDB7DEB726970FB6F894DEBF0FBECDBF92
:101140009E838D831C821B821DC08D818A838D812D
:101150009E81892F99278983698185E00E94E70014
:101160006A8186E00E94E70060E087E00E94E70075
:101170008D819E814E969E838D838B819C8101966D
:101180009C838B838B819C8188309105F0F226961D
:101190000FB6F894DEBF0FBECDBFDF91CF9108959B
:1011A000CF93DF93CDB7DEB727970FB6F894DEBFA6
:1011B0000FBECDBF9E838D836F831C821B8223C095
:1011C0008D818A838D819E81892F99278983698169
:1011D00085E00E94E7006A8186E00E94E7008F8137
:1011E0009927FC01E35DFE4F8081682F87E00E9414
:1011F000E7008D819E814E969E838D838B819C819D
:1012000001969C838B838B819C8188309105C0F2F1
:1012100027960FB6F894DEBF0FBECDBFDF91CF91FA
:101220000895CF93DF93CDB7DEB726970FB6F89426
:10123000DEBF0FBECDBF8091A8039091A90326E128
:1012400030E0B9010E940711CB019E838D838D810F
:101250009E8199230CF452C08D819E812AE030E05A
:10126000B9010E940711CB018A838D819E812AE0FA
:1012700030E0B9010E9407118983898186958983AD
:101280008A81282F332787E090E0AC01421B530B63
:101290009A018EE190E0AC01249FC001259F900D42
:1012A000349F900D11240A969C838B8320910B010F
:1012B00030910C018B819C818217930761F08091A2
:1012C0000B0190910C010E94E1098B819C81698145
:1012D0000E94440A0AC0909108038981981729F056
:1012E0008B819C8169810E94440A898180930803D3
:1012F0008B819C8190930C0180930B018D819E8149
:1013000099230CF055C08D819E81909581959F4FBA
:101310009E838D838D819E812AE030E0B9010E94F9
:101320000711CB018A838D819E812AE030E0B901CB
:101330000E9407118983898186958C5F89838A81C0
:10134000282F33278EE190E0AC01249FC001259F18
:10135000900D349F900D112486509F4F9C838B835A
:1013600020910B0130910C018B819C818217930796
:1013700061F080910B0190910C010E94E1098B8139
:101380009C8169810E94440A0AC090910803898166
:10139000981729F08B819C8169810E94440A898178
:1013A000809308038B819C8190930C0180930B01A7
:1013B00026960FB6F894DEBF0FBECDBFDF91CF915A
:1013C0000895CF93DF93CDB7DEB726970FB6F89485
:1013D000DEBF0FBECDBF9E838D838D819E819C839A
:1013E0008B8318C08B818A838B819C81892F99275D
:1013F0008983698185E00E94E7006A8186E00E9416
:10140000E70060E087E00E94E7008B819C81019605
:101410009C838B838D819E819C01275F3F4F8B81B5
:101420009C8182179307F0F280910803282F3327BD
:10143000C901880F991F820F931FFC01EF5EFE4FB9
:1014400080818823C1F08D819E8182969C838B83CD
:101450008B818A838B819C81892F992789836981DC
:1014600085E00E94E7006A8186E00E94E70060E074
:1014700087E00E94E70026960FB6F894DEBF0FBE05
:10148000CDBFDF91CF910895CF93DF93CDB7DEB776
:1014900027970FB6F894DEBF0FBECDBF9E838D8316
:1014A0006F838D819E819C838B8324C08B818983F4
:1014B0008B819C81892F99278A836A8185E00E948C
:1014C000E700698186E00E94E7008F81282F33279B
:1014D000C901880F991F820F931FFC01E15FFE4F26
:1014E0008081682F87E00E94E7008B819C810196B4
:1014F0009C838B838D819E819C01275F3F4F8B81D5
:101500009C818217930790F28D819E8104969C8323
:101510008B838B8189838B819C81892F99278A83F7
:101520006A8185E00E94E700698186E00E94E70009
:101530008F81282F3327C901880F991F820F931F8E
:10154000FC01E05FFE4F8081682F87E00E94E7008A
:101550008F81282F3327C901880F991F820F931F6E
:10156000FC01EF5EFE4F8081882321F18D819E81F9
:1015700082969C838B838B8189838B819C81892F2D
:1015800099278A836A8185E00E94E700698186E065
:101590000E94E7008F81282F3327C901880F991FE8
:1015A000820F931FFC01EF5EFE4F8081682F87E062
:1015B0000E94E70027960FB6F894DEBF0FBECDBF9E
:1015C000DF91CF910895CF93DF93CDB7DEB760E081
:1015D00085E00E94E70063E886E00E94E70060E99A
:1015E00087E00E94E70060E085E00E94E70064E891
:1015F00086E00E94E70061E987E00E94E70060E082
:1016000085E00E94E70065E886E00E94E70062E965
:1016100087E00E94E70060E085E00E94E70066E85E
:1016200086E00E94E70063E987E00E94E70060E04F
:1016300085E00E94E70067E886E00E94E70064E931
:1016400087E00E94E70060E085E00E94E70068E82C
:1016500086E00E94E70065E987E00E94E70060E01D
:1016600085E00E94E70069E886E00E94E70066E9FD
:1016700087E00E94E70060E085E00E94E7006AE8FA
:1016800086E00E94E70067E987E00E94E70060E0EB
:1016900085E00E94E70061EA86E00E94E70068E9D1
:1016A00087E00E94E70060E085E00E94E70062EAD0
:1016B00086E00E94E70069E987E00E94E70060E0B9
:1016C00085E00E94E70063EA86E00E94E7006AE99D
:1016D00087E00E94E70060E085E00E94E70064EA9E
:1016E00086E00E94E7006BE987E00E94E70060E087
:1016F00085E00E94E70065EA86E00E94E7006CE969
:1017000087E00E94E70060E085E00E94E70066EA6B
:1017100086E00E94E7006DE987E00E94E70060E054
:1017200085E00E94E70067EA86E00E94E7006EE934
:1017300087E00E94E70060E085E00E94E70068EA39
:1017400086E00E94E7006FE987E00E94E70060E022
:1017500085E00E94E7006FEB86E00E94E70060EA08
:1017600087E00E94E70060E085E00E94E70060EC0F
:1017700086E00E94E70061EA87E00E94E70060E0FF
:1017800085E00E94E70061EC86E00E94E70062EAE3
:1017900087E00E94E70060E085E00E94E70062ECDD
:1017A00086E00E94E70063EA87E00E94E70060E0CD
:1017B00085E00E94E70063EC86E00E94E70064EAAF
:1017C00087E00E94E70060E085E00E94E70064ECAB
:1017D00086E00E94E70065EA87E00E94E70060E09B
:1017E00085E00E94E70065EC86E00E94E70066EA7B
:1017F00087E00E94E70060E085E00E94E70066EC79
:1018000086E00E94E70067EA87E00E94E70060E068
:1018100085E00E94E7006DED86E00E94E70068EA3F
:1018200087E00E94E70060E085E00E94E7006EED3F
:1018300086E00E94E70069EA87E00E94E70060E036
:1018400085E00E94E7006FED86E00E94E7006AEA0B
:1018500087E00E94E70060E085E00E94E70060EE1C
:1018600086E00E94E7006BEA87E00E94E70060E004
:1018700085E00E94E70061EE86E00E94E7006CEAE6
:1018800087E00E94E70060E085E00E94E70062EEEA
:1018900086E00E94E7006DEA87E00E94E70060E0D2
:1018A00085E00E94E70063EE86E00E94E7006EEAB2
:1018B00087E00E94E70060E085E00E94E70064EEB8
:1018C00086E00E94E7006FEA87E00E94E70060E0A0
:1018D00085E00E94E7006BEF86E00E94E70060EB86
:1018E00087E00E94E70060E085E00E94E7006CEF7F
:1018F00086E00E94E70061EB87E00E94E70060E07D
:1019000085E00E94E7006DEF86E00E94E70062EB51
:1019100087E00E94E70060E085E00E94E7006EEF4C
:1019200086E00E94E70063EB87E00E94E70060E04A
:1019300085E00E94E7006FEF86E00E94E70064EB1D
:1019400087E00E94E70061E085E00E94E70060E038
:1019500086E00E94E70065EB87E00E94E70061E017
:1019600085E00E94E70061E086E00E94E70066EB08
:1019700087E00E94E700DF91CF910895CF93DF9336
:10198000CDB7DEB764970FB6F894DEBF0FBECDBFFC
:1019900083E090E09C8B8B8B1A82198283E990E024
:1019A0009C838B8310920B03CFC08B899C89FC0195
:1019B000E45FFC4F80819927CD979A8B898B8B8927
:1019C0009C8901969C8B8B8B8B899C89FC01E45FA5
:1019D000FC4F80819927CD97988B8F878B899C8925
:1019E00001969C8B8B8B8B899C89FC01E45FFC4F5F
:1019F00080819927CD979E878D878B899C890196B9
:101A00009C8B8B8B8B899C89FC01E45FFC4F8081D4
:101A10009927CD979C878B878B899C8901969C8B76
:101A20008B8B89899A899C01220F331F220F331FC8
:101A30008F8598899595879595958795959587959F
:101A400095958795822B932B9A8789878F8598897F
:101A50008F7090709C0122953295307F3227207FC5
:101A600032278D859E859595879595958795822BAF
:101A7000932B98878F838D859E85837090709C01B2
:101A80000024369527950794369527950794322F8D
:101A9000202D8B859C85822B932B9E838D838B8120
:101AA0009C8101979C838B838B819C812FEF8F3F3F
:101AB000920709F44EC089819A819C018091F702B6
:101AC0009091F802F901E80FF91F898580838981D7
:101AD0009A8101969A8389838B819C8101979C834B
:101AE0008B838B819C812FEF8F3F920791F18981AE
:101AF0009A819C018091F7029091F802F901E80F18
:101B0000F91F8F81808389819A8101969A838983C5
:101B10008B819C8101979C838B838B819C812FEF90
:101B20008F3F9207B1F089819A819C018091F702E1
:101B30009091F802F901E80FF91F8D818083898166
:101B40009A8101969A8389838B819C81009709F001
:101B50002CCF64960FB6F894DEBF0FBECDBFDF91D9
:101B6000CF910895CF93DF93CDB7DEB7E9E2F0E0F0
:101B700082E28083E0E4F0E01082E0E2F0E082E2E2
:101B80008083ECE5F0E01082A2E3B0E0E2E3F0E075
:101B9000808181608C93A8E3B0E0E8E3F0E080818D
:101BA00084608C93EAE2F0E088E98083E0E4F0E08E
:101BB00086E88083EBE2F0E082EC8083E1E2F0E013
:101BC00088E98083ECE5F0E086E88083E2E2F0E0FB
:101BD00082EC8083DF91CF910895CF93DF93CDB7CF
:101BE000DEB721970FB6F894DEBF0FBECDBF898355
:101BF000EBE2F0E080819927807290700097C1F34A
:101C0000ECE2F0E08981808321960FB6F894DEBF84
:101C10000FBECDBFDF91CF910895CF93DF93CDB7A6
:101C2000DEB726970FB6F894DEBF0FBECDBF9E83FA
:101C30008D838D819E81DC01FD0101900020E9F7FB
:101C40003197CF018A1B9B0B9C838B831A8219824D
:101C50000FC029813A818D819E81F901E80FF91F1A
:101C600080810E94ED0D89819A8101969A838983F2
:101C700029813A818B819C818217930750F780914B
:101C8000F9020E94ED0D8091FA020E94ED0D269658
:101C90000FB6F894DEBF0FBECDBFDF91CF91089590
:101CA000CF93DF93CDB7DEB766970FB6F894DEBF5C
:101CB0000FBECDBF9E8B8D8B8D899E894AE050E0F3
:101CC0009E012F5F3F4FB9010E94D610CE010196B1
:101CD0000E940D0E66960FB6F894DEBF0FBECDBF04
:101CE000DF91CF910895CF93DF93CDB7DEB72297E1
:101CF0000FB6F894DEBF0FBECDBF8A8387E089831D
:101D00001FC08A81482F55278981282F332727FD17
:101D1000309581E090E0022E02C0880F991F0A944E
:101D2000E2F7842395231816190624F481E30E9410
:101D3000ED0D03C080E30E94ED0D89818150898300
:101D400089818823F4F68091F9020E94ED0D80913B
:101D5000FA020E94ED0D22960FB6F894DEBF0FBE78
:101D6000CDBFDF91CF9108951F920F920FB60F92C2
:101D700011242F933F938F939F93AF93BF93EF9330
:101D8000FF93CF93DF93CDB7DEB72297DEBFCDBFF2
:101D9000E3E2F0E080818093E8038091E8038D30F6
:101DA000D1F480910A038130B1F4A5E3B0E0E5E31A
:101DB000F0E08081877F8C9310920A0381E080930A
:101DC0000B038091A20399272091E803FC01E45FB3
:101DD000FC4F208348C080910A03282F33273A8381
:101DE000298389819A81009731F029813A812130B4
:101DF000310521F138C08091E803833271F480917C
:101E00000B03882351F481E080930A03A5E3B0E03B
:101E1000E5E3F0E0808188608C931092A20330911A
:101E2000A203832F99272091E803FC01E45FFC4F74
:101E30002083832F8F5F8093A20315C08091A2031C
:101E400099272091E803FC01E45FFC4F20838091F7
:101E5000A203863930F48091A2038F5F8093A2039E
:101E600002C010920A032296F894DEBFCDBFDF9124
:101E7000CF91FF91EF91BF91AF919F918F913F9142
:101E80002F910F900FBE0F901F901895CF93DF9357
:101E9000CDB7DEB76E970FB6F894DEBF0FBECDBFDD
:101EA0002091A8033091A903CE010B964AE050E09F
:101EB000BC01C9010E94D61080E4898384E48A832E
:101EC00080E38B831C82CE010B96DC01FD01019027
:101ED0000020E9F73197CF018A1B9B0B9E01255FFC
:101EE0003F4FAC01B901CE0101960E94C610CE0150
:101EF0000196DC01FD0101900020E9F731979F0177
:101F00002A1B3B0BCE010196820F931FFC0183E23B
:101F100090E091838083CE0101960E940D0E209166
:101F2000AA033091AB03CE010B964AE050E0BC010E
:101F3000C9010E94D61080E4898384E48A8381E306
:101F40008B831C82CE010B96DC01FD0101900020E9
:101F5000E9F73197CF018A1B9B0B9E01255F3F4F0D
:101F6000AC01B901CE0101960E94C610CE010196C6
:101F7000DC01FD0101900020E9F731979F012A1B48
:101F80003B0BCE010196820F931FFC0183E290E090
:101F900091838083CE0101960E940D0E2091B203A1
:101FA0003091B303CE010B964AE050E0BC01C90169
:101FB0000E94D61080E4898388E68A838DE38B8330
:101FC0001C82CE010B96DC01FD0101900020E9F797
:101FD0003197CF018A1B9B0B9E01255F3F4FAC01C0
:101FE000B901CE0101960E94C610CE010196DC0116
:101FF000FD0101900020E9F731979F012A1B3B0B5F
:10200000CE010196820F931FFC0183E290E0918341
:102010008083CE0101960E940D0E2091BA0330916B
:10202000BB03CE010B964AE050E0BC01C9010E94FF
:10203000D61080E4898386E58A838CE68B831C82B4
:10204000CE010B96DC01FD0101900020E9F73197EC
:10205000CF018A1B9B0B9E01255F3F4FAC01B9014D
:10206000CE0101960E94C610CE010196DC01FD0151
:1020700001900020E9F731979F012A1B3B0BCE010D
:102080000196820F931FFC0183E290E0918380838D
:10209000CE0101960E940D0E20910403309105039C
:1020A000CE010B964AE050E0BC01C9010E94D61057
:1020B00080E4898386E58A8381E48B831C82CE0158
:1020C0000B96DC01FD0101900020E9F73197CF016B
:1020D0008A1B9B0B9E01255F3F4FAC01B901CE01CE
:1020E00001960E94C610CE010196DC01FD0101900F
:1020F0000020E9F731979F012A1B3B0BCE01019687
:10210000820F931FFC0183E290E091838083CE01D4
:1021100001960E940D0E6E960FB6F894DEBF0FBEAC
:10212000CDBFDF91CF910895CF93DF93CDB7DEB7C9
:10213000A5E3B0E0E5E3F0E0908182E089278C93AD
:10214000DF91CF910895CF93DF93CDB7DEB7809124
:1021500003038130C1F480910203813051F4A5E37F
:10216000B0E0E5E3F0E080818E7F8C931092020373
:102170000AC0A5E3B0E0E5E3F0E0808181608C93E4
:1021800081E080930203DF91CF910895FB01DC0190
:102190000D900020E9F711974150504028F0019030
:1021A00000200D92C9F708951C920895FB019F012C
:1021B000E8944230C4F04532B4F44A3029F497FB35
:1021C0001EF4909581959F4F642F77270E941A11D6
:1021D000805D8A330CF0895D8193CB010097A1F774
:1021E00016F45DE251931082C9010C94F710DC01E2
:1021F000FC0101900020E9F73297AE17BF0730F4D9
:102200007C916081708331976D93F7CF089597FB30
:10221000092E07260AD077FD04D00CD006D0002066
:102220001AF4709561957F4F0895F6F79095819512
:102230009F4F0895AA1BBB1B51E107C0AA1FBB1FDC
:10224000A617B70710F0A61BB70B881F991F5A9542
:0C225000A9F780959095BC01CD01089580
:10225C0001125A2C294400000A3100230023005497
:10226C0064665363655262005161005060005060B7
:10227C00005161005262005363655464666768697B
:10228C006A6B6B6A696867555555555555400155CC
:10229C002AA8152AAA85280AA12852A52854A828B4
:1022AC0055282869282869282855282854A82852F0
:1022BC00A5280AA12AAA852AA815400155555555C5
:1022CC005555555555555555555555555540000170
:1022DC004AAAA82AAAA828000128555528555528E5
:1022EC0000552AA8552AA855280055285555285573
:1022FC00552800012AAAA84AAAA8400001555555FC
:10230C00555555555555555555555555555000150B
:10231C004AAA852AAAA12800A82855282855282881
:10232C0000A82AAAA12AAA8528001528555528559F
:10233C0055285555285555285555415555555555DC
:10234C005555555555555555415554281552558586
:10235C0049416125285895285655415555415555A3
:10236C00285555285555285555285555285555281F
:10237C0055552855552855552855552855555555B5
:10238C0055555555555555955556255558495561DD
:10239C0052558554961555285555415555555555F5
:1023AC0055555555555555555555555555555555D1
:1023BC0055555555555555555555555555555555C1
:1023CC0055555555555555555555555555555555B1
:1023DC005555559555562555584955615255855461
:1023EC0096155528555541555555555555555555D1
:1023FC005555555555555555555555555555555581
:10240C005555555555555555555555555555555570
:10241C005555555555555555555555555555559520
:10242C00555625555849556152558554961555287C
:10243C005555415555555555555555555555555554
:0C244C0055555555555555A6030D0A0071
:00000001FF
